:020000040000FA
:0408000034EF0BF0D6
:1008100003B275EF05F0F2B493EF05F09EB09BEFD5
:1008200005F09EB2A3EF05F0F2A81AEF04F0F2B2C1
:1008300025EF04F0F2A620EF04F0F2B022EF04F06E
:10084000E3EF0AF0F296F290FF00CD90F2929EA0B4
:100850002FEF04F00101533F2FEF04F0542BAEC1F2
:10086000B2F1AFC1B3F1B0C1B4F1B1C1B5F1AAC138
:10087000AEF1ABC1AFF1ACC1B0F1ADC1B1F1A6C148
:10088000AAF1A7C1ABF1A8C1ACF1A9C1ADF1A2C158
:10089000A6F1A3C1A7F1A4C1A8F1A5C1A9F19EC168
:1008A000A2F19FC1A3F1A0C1A4F1A1C1A5F19AC178
:1008B0009EF19BC19FF19CC1A0F19DC1A1F196C188
:1008C0009AF197C19BF198C19CF199C19DF1CECF4E
:1008D00096F1CFCF97F153C198F154C199F1CF6AF6
:1008E000CE6A0101536B546B9E90CD800FBC0F8E6E
:1008F0000FBA7EEF04F00F8AE3EF0AF00F8C0FBE01
:10090000BAEF04F096C19AF197C19BF198C19CF19E
:1009100099C19DF19AC19EF19BC19FF19CC1A0F12B
:100920009DC1A1F19EC1A2F19FC1A3F1A0C1A4F1FB
:10093000A1C1A5F1A2C1A6F1A3C1A7F1A4C1A8F1CB
:10094000A5C1A9F1A6C1AAF1A7C1ABF1A8C1ACF19B
:10095000A9C1ADF1AAC1AEF1ABC1AFF1ACC1B0F16B
:10096000ADC1B1F1AEC1B2F1AFC1B3F1B0C1B4F13B
:10097000B1C1B5F101015E6B5F6B606B616B96514C
:100980005E2797515F2398516023995161239A51B3
:100990005E279B515F239C5160239D5161239E5193
:1009A0005E279F515F23A0516023A1516123A25173
:1009B0005E27A3515F23A4516023A5516123A65153
:1009C0005E27A7515F23A8516023A9516123AA5133
:1009D0005E27AB515F23AC516023AD516123AE5113
:1009E0005E27AF515F23B0516023B1516123B251F3
:1009F0005E27B3515F23B4516023B5516123D89072
:100A00000101613360335F335E33D890010161339C
:100A100060335F335E33D8900101613360335F33FD
:100A20005E3300C10CF101C10DF102C10EF103C131
:100A30000FF104C110F105C111F106C112F107C196
:100A400013F108C114F109C115F10AC116F10BC166
:100A500017F134C135F111B839EF05F00101620E1B
:100A6000046F010E056F000E066F000E076F42EF58
:100A700005F00101A70E046F020E056F000E066F50
:100A8000000E076F5EC100F15FC101F160C102F1AC
:100A900061C103F1BEEC24F003BF51EF05F011B6C4
:100AA000108C11A059EF05F010BA59EF05F00F8026
:100AB000108A0CC100F10DC101F10EC102F10FC18C
:100AC00003F110C104F111C105F112C106F113C106
:100AD00007F114C108F115C109F116C10AF117C1D6
:100AE0000BF135C134F1E3EF0AF00392ABB2AB98EE
:100AF000AB88030103EE00F080517F0BE92604C0B0
:100B0000EFFF802B8151805D700BD8A48B82000099
:100B10008051815D700BD8A48B9281518019D8B41B
:100B20000790E3EF0AF0F2940101453FE3EF0AF08A
:100B3000462BE3EF0AF09E900101533FE3EF0AF0EA
:100B4000542BE3EF0AF09E9211B815EF08F0040061
:100B500062A1ABEF05F08BB4B5EF05F010ACB5EFCB
:100B600005F08B84109CB6EF05F08B94077C07ACE6
:100B7000D1EF05F0C274C2B4CBEF05F0C3CFB3F52B
:100B8000C4CFB4F50501D890B433B333D890B4339F
:100B9000B333D2EF05F0C3CF55F1C4CF56F1D2EF46
:100BA00005F0C28207B43FEF06F047C14BF148C1E0
:100BB0004CF149C14DF14AC14EF15EC162F15FC1D4
:100BC00063F160C164F161C165F196C1B6F197C18D
:100BD000B7F198C1B8F199C1B9F19AC1BAF19BC105
:100BE000BBF19CC1BCF19DC1BDF19EC1BEF19FC1D5
:100BF000BFF1A0C1C0F1A1C1C1F1A2C1C2F1A3C1A5
:100C0000C3F1A4C1C4F1A5C1C5F1A6C1C6F1A7C174
:100C1000C7F1A8C1C8F1A9C1C9F1AAC1CAF1ABC144
:100C2000CBF1ACC1CCF1ADC1CDF1AEC1CEF1AFC114
:100C3000CFF1B0C1D0F1B1C1D1F1B2C1D2F1B3C1E4
:100C4000D3F1B4C1D4F1B5C1D5F1B3C5B5F5B4C5CF
:100C5000B6F5B5C5B7F5B6C5B8F5010155515B2771
:100C600056515C23E86A5D230E2E3FEF06F05CC10F
:100C700057F15DC158F15B6B5C6B5D6B078E0201D8
:100C8000002FE3EF0AF03C0E006F00C10CF101C130
:100C90000DF102C10EF103C10FF104C110F105C144
:100CA00011F106C112F107C113F108C114F109C114
:100CB00015F10AC116F10BC117F134C135F1050167
:100CC0002F51000AD8B410EF07F005012F51010A87
:100CD000D8B49AEF06F005012F51020AD8B4DBEF21
:100CE00006F005012F51030AD8B4DBEF06F0050129
:100CF0002F51040AD8B4DBEF06F005012F51050A85
:100D0000D8B4DBEF06F005012F51060AD8B4DBEFAB
:100D100006F005012F51070AD8B4DBEF06F00501F4
:100D20002F51320AD8B498EF06F02F6B10EF07F06E
:100D300010EF07F005015367A5EF06F05467A5EF24
:100D400006F05567A5EF06F05667A9EF06F010EF1D
:100D500007F057C500F158C501F159C502F15AC550
:100D600003F10101010E046F000E056F000E066F06
:100D7000000E076FBEEC24F000C157F501C158F515
:100D800002C159F503C15AF50067CEEF06F00167BD
:100D9000CEEF06F00267CEEF06F0036710EF07F024
:100DA00053C557F554C558F555C559F556C55AF5A7
:100DB0000F8810EF07F005013067E1EF06F010EF44
:100DC00007F00FBEF6EF06F010A0FBEF06F00101F2
:100DD0004767F2EF06F04867F2EF06F04967F2EF77
:100DE00006F04A67F6EF06F0FBEF06F007AEFBEF02
:100DF00006F00DEF07F00501312F10EF07F03C0E64
:100E0000316F302F10EF07F00101000E626FE00E1E
:100E1000636FA50E646F010E656F0501306B0F885F
:100E20000501626B33B716EF07F062810CC100F168
:100E30000DC101F10EC102F10FC103F110C104F1A6
:100E400011C105F112C106F113C107F114C108F176
:100E500015C109F116C10AF117C10BF135C134F101
:100E600000C10CF101C10DF102C10EF103C10FF17E
:100E700004C110F105C111F106C112F107C113F14E
:100E800008C114F109C115F10AC116F10BC117F11E
:100E900034C135F101018A6755EF07F08B6755EFD3
:100EA00007F08C6755EF07F08D6759EF07F089EF72
:100EB00007F08EC100F18FC101F190C102F191C123
:100EC00003F10101010E046F000E056F000E066FA5
:100ED000000E076FBEEC24F000C18EF101C18FF14E
:100EE00002C190F103C191F100677EEF07F0016745
:100EF0007EEF07F002677EEF07F0036789EF07F0E8
:100F00008AC18EF18BC18FF18CC190F18DC191F1AD
:100F10000F80D57ED5BE6BD0D6CF47F1D7CF48F165
:100F200045C149F1E86AE8CF4AF111B6108C10903A
:100F300047C100F148C101F149C102F14AC103F1C1
:100F400001010A0E046F000E056F000E066F000E01
:100F5000076FBEEC24F003AF1080010154A7BDEF72
:100F600007F00F9A0F9C0F9E0101000E5E6F600E3E
:100F70005F6F3D0E606F080E616F010147BFCDEFDF
:100F800007F04867CDEF07F04967CDEF07F04A67F4
:100F9000CDEF07F0F288F2EF07F0F2985E6B5F6B2F
:100FA000606B616B966B976B986B996B9A6B9B6B95
:100FB0009C6B9D6B9E6B9F6BA06BA16BA26BA36BDD
:100FC000A46BA56BA66BA76BA86BA96BAA6BAB6B8D
:100FD000AC6BAD6BAE6BAF6BB06BB16BB26BB36B3D
:100FE000B46BB56BD76AD66A0101456B466B0CC111
:100FF00000F10DC101F10EC102F10FC103F110C1E9
:1010000004F111C105F112C106F113C107F114C1B8
:1010100008F115C109F116C10AF117C10BF135C16B
:1010200034F1E3EF0AF0E3EF0AF00201002F4CEF96
:101030000AF0D59ED6CF47F1D7CF48F145C149F147
:10104000E86AE8CF4AF1D76AD66A0101456B466B78
:10105000D58E00C10CF101C10DF102C10EF103C129
:101060000FF104C110F105C111F106C112F107C160
:1010700013F108C114F109C115F10AC116F10BC130
:1010800017F134C135F10FA0109A11B853EF08F0E1
:101090000101620E046F010E056F000E066F000E57
:1010A000076F5CEF08F00101A70E046F020E056FD9
:1010B000000E066F000E076F47C100F148C101F135
:1010C00049C102F14AC103F1BEEC24F003BF6DEF48
:1010D00008F011B6108C11B00F800CC100F10DC1D9
:1010E00001F10EC102F10FC103F110C104F111C1F0
:1010F00005F112C106F113C107F114C108F115C1C0
:1011000009F116C10AF117C10BF135C134F1020121
:101110003C0E006F00C10CF101C10DF102C10EF1D6
:1011200003C10FF104C110F105C111F106C112F1A3
:1011300007C113F108C114F109C115F10AC116F173
:101140000BC117F134C135F105012F51000AD8B494
:1011500055EF09F005012F51010AD8B4DFEF08F06F
:1011600005012F51020AD8B420EF09F005012F51D3
:10117000030AD8B420EF09F005012F51040AD8B4AE
:1011800020EF09F005012F51050AD8B420EF09F02E
:1011900005012F51060AD8B420EF09F005012F519F
:1011A000070AD8B420EF09F005012F51320AD8B44C
:1011B000DDEF08F02F6B55EF09F055EF09F0050151
:1011C0005367EAEF08F05467EAEF08F05567EAEF73
:1011D00008F05667EEEF08F055EF09F057C500F13B
:1011E00058C501F159C502F15AC503F10101010EBB
:1011F000046F000E056F000E066F000E076FBEEC49
:1012000024F000C157F501C158F502C159F503C1D9
:101210005AF5006713EF09F0016713EF09F0026751
:1012200013EF09F0036755EF09F053C557F554C59F
:1012300058F555C559F556C55AF50F8855EF09F0BB
:101240000501306726EF09F055EF09F00FBE3BEFBF
:1012500009F010A040EF09F00101476737EF09F0EE
:10126000486737EF09F0496737EF09F04A673BEF06
:1012700009F040EF09F007AE40EF09F052EF09F036
:101280000501312F55EF09F03C0E316F302F55EF2E
:1012900009F00101000E626FE00E636FA50E646F2E
:1012A000010E656F0501306B0F880501626B33B766
:1012B0005BEF09F062810CC100F10DC101F10EC1BB
:1012C00002F10FC103F110C104F111C105F112C106
:1012D00006F113C107F114C108F115C109F116C1D6
:1012E0000AF117C10BF135C134F100C10CF101C194
:1012F0000DF102C10EF103C10FF104C110F105C1DE
:1013000011F106C112F107C113F108C114F109C1AD
:1013100015F10AC116F10BC117F134C135F1010104
:101320008A679AEF09F08B679AEF09F08C679AEF5A
:1013300009F08D679EEF09F0CEEF09F08EC100F144
:101340008FC101F190C102F191C103F10101010EC0
:10135000046F000E056F000E066F000E076FBEECE7
:1013600024F000C18EF101C18FF102C190F103C1DF
:1013700091F10067C3EF09F00167C3EF09F002675D
:10138000C3EF09F00367CEEF09F08AC18EF18BC17C
:101390008FF18CC190F18DC191F10F80109047C1F8
:1013A00000F148C101F149C102F14AC103F1010153
:1013B0000A0E046F000E056F000E066F000E076F19
:1013C000BEEC24F003AF1080010154A7F4EF09F044
:1013D0000F9A0F9C0F9E0101000E5E6F600E5F6FF3
:1013E0003D0E606F080E616F47C100F148C101F109
:1013F00049C102F14AC103F10101140E046F050E47
:10140000056F000E066F000E076FBEEC24F003AFF1
:101410000DEF0AF0F28832EF0AF0F2985E6B5F6B24
:10142000606B616B966B976B986B996B9A6B9B6B10
:101430009C6B9D6B9E6B9F6BA06BA16BA26BA36B58
:10144000A46BA56BA66BA76BA86BA96BAA6BAB6B08
:10145000AC6BAD6BAE6BAF6BB06BB16BB26BB36BB8
:10146000B46BB56B0CC100F10DC101F10EC102F1FD
:101470000FC103F110C104F111C105F112C106F150
:1014800013C107F114C108F115C109F116C10AF120
:1014900017C10BF135C134F104008BB457EF0AF0DA
:1014A00010AC57EF0AF08B84109C58EF0AF08B9425
:1014B000077C07AC73EF0AF0C274C2B46DEF0AF098
:1014C000C3CFB3F5C4CFB4F50501D890B433B3336B
:1014D000D890B433B33374EF0AF0C3CF55F1C4CF0F
:1014E00056F174EF0AF0C28207B4E1EF0AF047C187
:1014F0004BF148C14CF149C14DF14AC14EF15EC1B9
:1015000062F15FC163F160C164F161C165F196C1CF
:10151000B6F197C1B7F198C1B8F199C1B9F19AC1C3
:10152000BAF19BC1BBF19CC1BCF19DC1BDF19EC193
:10153000BEF19FC1BFF1A0C1C0F1A1C1C1F1A2C163
:10154000C2F1A3C1C3F1A4C1C4F1A5C1C5F1A6C133
:10155000C6F1A7C1C7F1A8C1C8F1A9C1C9F1AAC103
:10156000CAF1ABC1CBF1ACC1CCF1ADC1CDF1AEC1D3
:10157000CEF1AFC1CFF1B0C1D0F1B1C1D1F1B2C1A3
:10158000D2F1B3C1D3F1B4C1D4F1B5C1D5F1B3C572
:10159000B5F5B4C5B6F5B5C5B7F5B6C5B8F501012D
:1015A00055515B2756515C23E86A5D230E2EE1EF0F
:1015B0000AF05CC157F15DC158F15B6B5C6B5D6B10
:1015C000078EE3EF0AF002C0E0FF005001C0D8FF31
:1015D0001000A6B2E9EF0AF00CC0A9FF0BC0A8FFEB
:1015E000A69EA69CA684F29E550EA76EAA0EA76E76
:1015F000A682F28EA694A6B2FBEF0AF00C2A120085
:10160000A96EA69EA69CA680A8500C2A12000401D2
:101610002C0E826F24EC0EF0B9EC25F00C5000EC8F
:101620000BF0E8CF00F10C5000EC0BF0E8CF01F12B
:1016300001AF20EF0BF00101FF0E026FFF0E036FF1
:101640005CEC25F029672CEF0BF00401200E826F73
:1016500024EC0EF031EF0BF004012D0E826F24EC20
:101660000EF086EC23F01200076A0F6A106A116A06
:101670000F010D0EC16E860EC06E030EC26E0F01FD
:10168000680E896E130E926E080E8A6EF30E936EBC
:101690008B6A900E946EC80E00EC0BF0E8CFE8FF5A
:1016A0001098E8A0108810A805D00E0E166E8E0EA9
:1016B000176E04D00F0E166E8F0E176E38EC26F0D4
:1016C000F18EF19EFC0E00EC0BF0E8CF0BF00BA0BE
:1016D00011800BA211820BA411840BA611860BA8FA
:1016E00011880BAA118A0E6A01015B6B5C6B5D6B42
:1016F000576B586BF29A0101476B486B496B4A6B09
:101700004B6B4C6B4D6B4E6B4F6B506B516B526B0D
:10171000456B466BD76AD66A0F01280ED56EF28AE2
:101720009D90B00ECD6E01015E6B5F6B606B616B67
:10173000626B636B646B656B666B676B686B696B25
:10174000536B546BCF6ACE6A0F9A0F9C0F9E9D808D
:10175000760ECA6E9D8202013C0E006FCC6A160E98
:1017600000EC0BF0E8CF00F1170E00EC0BF0E8CF27
:1017700001F1180E00EC0BF0E8CF02F1190E00ECAD
:101780000BF0E8CF03F1010103AFE1EF0BF0B9EC8F
:1017900025F0160E0C6E00C10BF0E9EC0AF0170EE6
:1017A0000C6E01C10BF0E9EC0AF0180E0C6E02C1D0
:1017B0000BF0E9EC0AF0190E0C6E03C10BF0E9EC2A
:1017C0000AF000C18AF101C18BF102C18CF103C1A1
:1017D0008DF100C18EF101C18FF102C190F103C101
:1017E00091F11A0E00EC0BF0E8CF00F11B0E00ECAB
:1017F0000BF0E8CF01F11C0E00EC0BF0E8CF02F18A
:101800001D0E00EC0BF0E8CF03F1010103AF37EF41
:101810000CF0B9EC25F01A0E0C6E00C10BF0E9ECDF
:101820000AF01B0E0C6E01C10BF0E9EC0AF01C0E65
:101830000C6E02C10BF0E9EC0AF01D0E0C6E03C138
:101840000BF0E9EC0AF01A0E00EC0BF0E8CF00F117
:101850001B0E00EC0BF0E8CF01F11C0E00EC0BF0BE
:10186000E8CF02F11D0E00EC0BF0E8CF03F100C150
:1018700092F101C193F102C194F103C195F1240EDB
:10188000AC6E900EAB6E240EAC6E080EB86E000EF1
:10189000B06E1F0EAF6E0401806B816B0F01900E56
:1018A000AB6E0F019D8A0301806B816BC26B8B92C3
:1018B000C0EC2AF0C0EC2AF01CEC2CF09FEC28F0D5
:1018C000200E00EC0BF0E8CF2FF505012F51FF0A99
:1018D000D8A472EF0CF02F6B200E0C6E2FC50BF0FE
:1018E000E9EC0AF00501010E306F3C0E316F250E58
:1018F00000EC0BF0E8CF00F1260E00EC0BF0E8CF87
:1019000001F1270E00EC0BF0E8CF02F1280E00ECFD
:101910000BF0E8CF03F1010103AFA9EF0CF0B9EC34
:1019200025F0250E0C6E00C10BF0E9EC0AF0260E36
:101930000C6E01C10BF0E9EC0AF0270E0C6E02C12F
:101940000BF0E9EC0AF0280E0C6E03C10BF0E9EC89
:101950000AF000C153F501C154F502C155F503C1A8
:1019600056F500C157F501C158F502C159F503C13B
:101970005AF5290E00EC0BF0E8CF5BF505015C5140
:101980005B5DD8A05BC55CF505012F51020A0EE135
:1019900081B8D6EF0CF005015C2FD3EF0CF05BC5DE
:1019A0005CF5D6EF0CF081BA5BEF2CF0210E00EC69
:1019B0000BF0E8CF00F1220E00EC0BF0E8CF01F1C4
:1019C000230E00EC0BF0E8CF02F1240E00EC0BF03C
:1019D000E8CF03F1010103AF1CEF0DF0B9EC25F0E6
:1019E000210E0C6E00C10BF0E9EC0AF0220E0C6E19
:1019F00001C10BF0E9EC0AF0230E0C6E02C10BF0F2
:101A0000E9EC0AF0240E0C6E03C10BF0E9EC0AF0CD
:101A1000210E00EC0BF0E8CF00F1220E00EC0BF0F1
:101A2000E8CF01F1230E00EC0BF0E8CF02F1240E19
:101A300000EC0BF0E8CF03F100C15DF501C15EF5EC
:101A400002C15FF503C160F5E7EC27F0E9EC26F091
:101A500041EC26F005012F51030A12E005012F5138
:101A6000040A1DE005012F51050A24E005012F514C
:101A7000060A32E005012F51070A38E07FEF0DF02A
:101A8000ACC500F101010F0E001701010051000A61
:101A900036E001010051050A32E07CEF0DF0ACC5E3
:101AA00000F101010F0E001701010051000A27E0AB
:101AB0007CEF0DF00501AC51000A21E00501AC51AD
:101AC000150A1DE00501AC51300A19E00501AC51C1
:101AD000450A15E07CEF0DF00501AC51000A0FE05E
:101AE0000501AC51300A0BE07CEF0DF00501AC5163
:101AF000000A05E07CEF0DF081BA5BEF2CF0079057
:101B00000001F28EF28C07B007EF22F00FB0ADEFBC
:101B10001CF00FB863EF16F00301805181197F0BA1
:101B2000D8B407EF22F013EE00F081517F0BE126CD
:101B3000812BE7CFE8FFE00BD8B407EF22F023EECC
:101B400082F0C2513F0BD926E7CFDFFFC22BDF5017
:101B5000780AD8A407EF22F007808EC100F18FC168
:101B600001F190C102F191C103F10101040E046F72
:101B7000000E056F000E066F000E076FBEEC24F01E
:101B800000AFCCEF0DF00101030E8E6F000E8F6FD2
:101B9000000E906F000E916F03018251720AD8B44B
:101BA000ADEF1CF08251520AD8B4ADEF1CF0825157
:101BB000750AD8B4ADEF1CF08251630AD8B4C1EFF6
:101BC0001EF08251690AD8B45AEF19F082517A0A8C
:101BD000D8B46DEF1AF08251490AD8B4F9EF18F071
:101BE0008251500AD8B417EF18F08251700AD8B455
:101BF0005AEF18F08251540AD8B485EF18F0825188
:101C0000740AD8B4CBEF18F082516D0AD8B429EF1A
:101C10000FF082514D0AD8B442EF0FF08251730A8F
:101C2000D8B4DDEF1BF08251530AD8B442EF1CF058
:101C300082514C0AD8B4D1EF0FF08251590AD8B46E
:101C400038EF0EF0F8EF1EF0040114EE00F08051B2
:101C50007F0BE12682C4E7FF802B120004010D0EEA
:101C6000826F24EC0EF00A0E826F24EC0EF012004C
:101C7000FC0E00EC0BF0E8CF0BF003018351520A8D
:101C8000D8B487EF0EF003018351720AD8B48AEFFB
:101C90000EF003018351500AD8B48DEF0EF003010A
:101CA0008351700AD8B490EF0EF003018351550AA6
:101CB000D8B493EF0EF003018351750AD8B496EFB0
:101CC0000EF0030183514C0AD8B499EF0EF00301D2
:101CD00083516C0AD8B49CEF0EF003018351430A80
:101CE000D8B49FEF0EF003018351630AD8B4A2EF7A
:101CF0000EF003018351440AD8B4A5EF0EF003019E
:101D00008351640AD8B4A8EF0EF0B1EF0EF00B9037
:101D1000ABEF0EF00B80ABEF0EF00B92ABEF0EF0D3
:101D20000B82ABEF0EF00B94ABEF0EF00B84ABEF2E
:101D30000EF00B96ABEF0EF00B86ABEF0EF00B98A0
:101D4000ABEF0EF00B88ABEF0EF00B9AABEF0EF093
:101D50000B8AABEF0EF0FC0E0C6E0BC00BF0E9EC37
:101D60000AF00401590E826F24EC0EF011901192CA
:101D7000119411961198119AFC0E00EC0BF0E8CF1B
:101D80000BF00BA011800BA211820BA411840BA6E7
:101D900011860BA811880BAA118A11A0D7EF0EF09B
:101DA0000401520E826F24EC0EF0DCEF0EF0040101
:101DB000720E826F24EC0EF011A6E6EF0EF0040115
:101DC0004C0E826F24EC0EF0EBEF0EF004016C0E63
:101DD000826F24EC0EF011A8F5EF0EF00401430E13
:101DE000826F24EC0EF0FAEF0EF00401630E826FA6
:101DF00024EC0EF011A204EF0FF00401500E826FDC
:101E000024EC0EF009EF0FF00401700E826F24EC49
:101E10000EF011A413EF0FF00401550E826F24ECA5
:101E20000EF018EF0FF00401750E826F24EC0EF027
:101E300011AA22EF0FF00401440E826F24EC0EF081
:101E400027EF0FF00401640E826F24EC0EF0F6EF22
:101E50001EF004016D0E826F24EC0EF0030183511D
:101E6000300AD8B481EF0FF003018351310AD8B49E
:101E700094EF0FF003018351320AD8B4A7EF0FF0AB
:101E8000F8EF1EF004014D0E826F24EC0EF0FAEC18
:101E900025F084C331F185C332F186C333F10101EA
:101EA000296B07EC26F07EEC25F003018351300A04
:101EB000D8B469EF0FF003018351310AD8B471EF40
:101EC0000FF003018351320AD8B479EF0FF0F8EF25
:101ED0001EF0FD0E0C6E00C10BF0E9EC0AF081EF74
:101EE0000FF0FE0E0C6E00C10BF0E9EC0AF094EF5F
:101EF0000FF0FF0E0C6E00C10BF0E9EC0AF0A7EF3B
:101F00000FF00401300E826F24EC0EF004012C0E51
:101F1000826F24EC0EF0B9EC25F0FD0E00EC0BF016
:101F2000E8CF00F1B8EF0FF00401310E826F24EC1E
:101F30000EF004012C0E826F24EC0EF0B9EC25F0AB
:101F4000FE0E00EC0BF0E8CF00F1B8EF0FF004014B
:101F5000320E826F24EC0EF0B9EC25F004012C0E49
:101F6000826F24EC0EF0FF0E00EC0BF0E8CF00F1D6
:101F70005CEC25F031C182F40401300E822724ECA0
:101F80000EF032C182F40401300E822724EC0EF0F0
:101F900033C182F40401300E822724EC0EF0F6EFF8
:101FA0001EF003018351300AD8B43CEF13F0030153
:101FB0008351310AD8B469EF14F003018351320A16
:101FC000D8B4D7EF14F003018351330AD8B4E7EF44
:101FD00014F003018351340AD8B4F7EF14F003016D
:101FE0008351350AD8B468EF16F003018351360ADD
:101FF000D8B496EF16F003018351370AD8B49EEF98
:1020000012F003018351460AD8B4BCEF15F0030166
:1020100083514D0AD8B417EF11F0030183516D0AB3
:10202000D8B431EF11F0030183515A0AD8B4E3EF69
:1020300013F003018351490AD8B496EF17F0030156
:102040008351500AD8B4C8EF16F003018351540AE3
:10205000D8B441EF17F003018351630AD8B451EFAC
:1020600011F003018351430AD8B449EF12F0030180
:102070008351730AD8B44FEF11F003018351610A01
:10208000D8B464EF10F003018351650AD8B48CEF23
:1020900013F003018351450AD8B49AEF13F00301FA
:1020A0008351620AD8B4A8EF13F003018351420AA6
:1020B000D8B4B6EF13F003018351760AD8B4C4EF55
:1020C00013F0D8A4F8EF1EF004014C0E826F24EC3C
:1020D0000EF00401610E826F24EC0EF0E9EC26F0A4
:1020E00004012C0E826F24EC0EF0B9EC25F0ABC588
:1020F00000F101015CEC25F031C182F40401300EE5
:10210000822724EC0EF032C182F40401300E8227C3
:1021100024EC0EF033C182F40401300E822724EC4B
:102120000EF004012C0E826F24EC0EF0B9EC25F0B9
:10213000ACC500F101015CEC25F031C182F4040171
:10214000300E822724EC0EF032C182F40401300EEE
:10215000822724EC0EF033C182F40401300E822772
:1021600024EC0EF004012C0E826F24EC0EF0B9EC7E
:1021700025F0ADC500F101015CEC25F031C182F420
:102180000401300E822724EC0EF032C182F40401E7
:10219000300E822724EC0EF033C182F40401300E9D
:1021A000822724EC0EF004012C0E826F24EC0EF03A
:1021B000B9EC25F0AEC500F101015CEC25F031C1B0
:1021C00082F40401300E822724EC0EF032C182F436
:1021D0000401300E822724EC0EF033C182F4040196
:1021E000300E822724EC0EF004012C0E826F24ECBA
:1021F0000EF0B9EC25F0B2C500F101015CEC25F060
:1022000031C182F40401300E822724EC0EF032C179
:1022100082F40401300E822724EC0EF033C182F4E4
:102220000401300E822724EC0EF0C4EF16F0FAEC15
:1022300025F084C333F107EC26F07EEC25F0200E68
:102240000C6E00C10BF0E9EC0AF000C12FF505019E
:102250002F51000A06E005012F51010A02E083EC2C
:1022600027F004014C0E826F24EC0EF004014D0E99
:10227000826F24EC0EF004012C0E826F24EC0EF021
:10228000B9EC25F02FC500F15CEC25F033C182F4E8
:102290000401300E822724EC0EF0C4EF16F05BEF41
:1022A0002CF004014C0E826F24EC0EF00401630E3E
:1022B000826F24EC0EF041EC26F004012C0E826FAC
:1022C00024EC0EF066EC11F0C4EF16F0B9EC25F03A
:1022D000B1C500F10101003B0F0E00175CEC25F0C9
:1022E00033C182F40401300E822724EC0EF0B1C514
:1022F00000F101010F0E010100175CEC25F033C164
:1023000082F40401300E822724EC0EF004012D0E1D
:10231000826F24EC0EF0B0C500F10101003B0F0EFE
:1023200000175CEC25F033C182F40401300E8227E3
:1023300024EC0EF0B0C500F101010F0E01010017F1
:102340005CEC25F033C182F40401300E822724ECCA
:102350000EF004012D0E826F24EC0EF0AFC500F1DB
:102360000101003B0F0E00175CEC25F033C182F435
:102370000401300E822724EC0EF0AFC500F10101FC
:102380000F0E010100175CEC25F033C182F404014B
:10239000300E822724EC0EF00401200E826F24EC14
:1023A0000EF0AEC500F10F0E010100175CEC25F038
:1023B00033C182F40401300E822724EC0EF00401B4
:1023C000200E826F24EC0EF0ADC500F10101010179
:1023D000003B0F0E00175CEC25F033C182F40401C2
:1023E000300E822724EC0EF0ADC500F101010F0E76
:1023F000010100175CEC25F033C182F40401300EBA
:10240000822724EC0EF004013A0E826F24EC0EF0C9
:10241000ACC500F10101003B0F0E00175CEC25F08C
:1024200033C182F40401300E822724EC0EF0ACC5D7
:1024300000F101010F0E010100175CEC25F033C122
:1024400082F40401300E822724EC0EF004013A0ECF
:10245000826F24EC0EF0ABC500F10101003B0F0EC2
:1024600000175CEC25F033C182F40401300E8227A2
:1024700024EC0EF0ABC500F101010F0E00175CEC6F
:1024800025F033C182F40401300E822724EC0EF0D3
:10249000120084C3E8FF0F0BE83AE8CFB1F585C31B
:1024A000E8FF0F0B0501B11387C3E8FF0F0BE83AF4
:1024B000E8CFB0F588C3E8FF0F0B0501B0138AC35E
:1024C000E8FF0F0BE83AE8CFAFF58BC3E8FF0F0B3F
:1024D0000501AF138DC3E8FF0F0BE8CFAEF58FC337
:1024E000E8FF0F0BE83AE8CFADF590C3E8FF0F0B1C
:1024F0000501AD1392C3E8FF0F0BE83AE8CFACF546
:1025000093C3E8FF0F0B0501AC1395C3E8FF0F0B56
:10251000E83AE8CFABF596C3E8FF0F0B0501AB1324
:102520009CEC26F004014C0E826F24EC0EF00401AA
:10253000430E826F24EC0EF05BEF11F00784040170
:102540004C0E826F24EC0EF00401370E826F24ECE7
:102550000EF004012C0E826F24EC0EF005012E51BA
:10256000130A06E005012E51170A0DE039EF13F0AA
:102570000101000E006F000E016F100E026F000EC1
:10258000036FCCEF12F00101000E006F000E016F1F
:10259000000E026F010E036F5CEC25F02AC182F47D
:1025A0000401300E822724EC0EF02BC182F40401CA
:1025B000300E822724EC0EF02CC182F40401300E80
:1025C000822724EC0EF02DC182F40401300E822704
:1025D00024EC0EF02EC182F40401300E822724EC8C
:1025E0000EF02FC182F40401300E822724EC0EF08D
:1025F00030C182F40401300E822724EC0EF031C188
:1026000082F40401300E822724EC0EF032C182F4F1
:102610000401300E822724EC0EF033C182F4040151
:10262000300E822724EC0EF004012C0E826F24EC75
:102630000EF00101100E006F000E016F000E026F10
:10264000000E036F5CEC25F031C182F40401300E02
:10265000822724EC0EF032C182F40401300E82276E
:1026600024EC0EF033C182F40401300E822724ECF6
:102670000EF00794C4EF16F007841CEC2CF0B9ECB4
:1026800025F02DC500F15CEC25F004014C0E826FA5
:1026900024EC0EF00401300E826F24EC0EF00401E5
:1026A0002C0E826F24EC0EF031C182F40401300E46
:1026B000822724EC0EF032C182F40401300E82270E
:1026C00024EC0EF033C182F40401300E822724EC96
:1026D0000EF004012C0E826F24EC0EF0B9EC25F004
:1026E0002EC500F15CEC25F031C182F40401300EFE
:1026F000822724EC0EF032C182F40401300E8227CE
:1027000024EC0EF033C182F40401300E822724EC55
:102710000EF00794C4EF16F004014C0E826F24EC07
:102720000EF00401650E826F24EC0EF043EC28F0ED
:10273000C4EF16F004014C0E826F24EC0EF004017D
:10274000450E826F24EC0EF05AEC28F0C4EF16F020
:1027500004014C0E826F24EC0EF00401620E826FB5
:1027600024EC0EF088EC28F0C4EF16F004014C0EB7
:10277000826F24EC0EF00401420E826F24EC0EF006
:1027800071EC28F0C4EF16F004014C0E826F24ECBB
:102790000EF00401760E826F24EC0EF004012C0E74
:1027A000826F24EC0EF010A807D00401310E826F66
:1027B00024EC0EF0C4EF16F00401300E826F24EC0E
:1027C0000EF0C4EF16F004014C0E826F24EC0EF0F4
:1027D00004015A0E826F24EC0EF004012C0E826F5D
:1027E00024EC0EF01CEC2CF0B9EC25F005012E5178
:1027F000130A06E005012E51170A0DE014EF14F03C
:102800000101000E006F000E016F100E026F000E2E
:10281000036F14EF14F00101000E006F000E016F42
:10282000000E026F010E036F0101100E046F000E07
:10283000056F000E066F000E076FEFEC24F05CECE6
:1028400025F02AC182F40401300E822724EC0EF018
:102850002BC182F40401300E822724EC0EF02CC12F
:1028600082F40401300E822724EC0EF02DC182F494
:102870000401300E822724EC0EF02EC182F40401F4
:10288000300E822724EC0EF02FC182F40401300EAA
:10289000822724EC0EF030C182F40401300E82272E
:1028A00024EC0EF031C182F40401300E822724ECB6
:1028B0000EF032C182F40401300E822724EC0EF0B7
:1028C00033C182F40401300E822724EC0EF0C4EFF1
:1028D00016F0078404014C0E826F24EC0EF0040104
:1028E000310E826F24EC0EF004012C0E826F24EC6A
:1028F0000EF025C500F126C501F127C502F128C556
:1029000003F10101100E046F000E056F000E066F3B
:10291000000E076FEFEC24F05CEC25F02AC182F486
:102920000401300E822724EC0EF02BC182F4040146
:10293000300E822724EC0EF02CC182F40401300EFC
:10294000822724EC0EF02DC182F40401300E822780
:1029500024EC0EF02EC182F40401300E822724EC08
:102960000EF02FC182F40401300E822724EC0EF009
:1029700030C182F40401300E822724EC0EF031C104
:1029800082F40401300E822724EC0EF032C182F46E
:102990000401300E822724EC0EF033C182F40401CE
:1029A000300E822724EC0EF00794C4EF16F0078453
:1029B00004014C0E826F24EC0EF00401320E826F83
:1029C00024EC0EF076EC2AF00794C4EF16F007849E
:1029D00004014C0E826F24EC0EF00401330E826F62
:1029E00024EC0EF0D3EC2AF0079474EF14F0078473
:1029F00004014C0E826F24EC0EF00401340E826F41
:102A000024EC0EF004012C0E826F24EC0EF0FAEC94
:102A100025F084C32AF185C32BF186C32CF187C32B
:102A20002DF188C32EF189C32FF18AC330F18BC3F6
:102A300031F18CC332F18DC333F10101296B07EC05
:102A400026F07EEC25F0100E046F000E056F000ED0
:102A5000066F000E076FCFEC24F000C121F501C115
:102A600022F502C123F503C124F5CFEC2BF034C5C8
:102A7000ABF535C5ACF536C5ADF537C5AEF538C5E2
:102A8000AFF539C5B0F53AC5B1F566EC11F0040102
:102A90002C0E826F24EC0EF03BC500F13CC501F119
:102AA0003DC502F13EC503F10101000E046F000EA9
:102AB000056F010E066F000E076FEFEC24F05CEC63
:102AC00025F0296766EF15F06BEF15F004012D0E68
:102AD000826F24EC0EF030C182F40401300E8227A4
:102AE00024EC0EF031C182F40401300E822724EC74
:102AF0000EF004012E0E826F24EC0EF032C182F42F
:102B00000401300E822724EC0EF033C182F404015C
:102B1000300E822724EC0EF004012C0E826F24EC80
:102B20000EF0B9EC25F03FC500F140C501F122ECF3
:102B300020F004012C0E826F24EC0EF0B9EC25F08D
:102B400041C500F15CEC25F031C182F40401300E86
:102B5000822724EC0EF032C182F40401300E822769
:102B600024EC0EF033C182F40401300E822724ECF1
:102B70000EF00794C4EF16F0FAEC25F085C32AF1A5
:102B800086C32BF187C32CF188C32DF189C32EF1A5
:102B90008AC32FF18BC330F18CC331F18DC332F175
:102BA0008EC333F10101296B07EC26F07EEC25F092
:102BB0000101010E046F000E056F000E066F000E7E
:102BC000076FBEEC24F0100E046F000E056F000EB0
:102BD000066F000E076FCFEC24F000C129F501C18C
:102BE0002AF502C12BF503C12CF5FDEC29F00401F7
:102BF0004C0E826F24EC0EF00401460E826F24EC22
:102C00000EF004012C0E826F24EC0EF025C500F1AD
:102C100026C501F127C502F128C503F10101100EF7
:102C2000046F000E056F000E066F000E076FEFECCD
:102C300024F05CEC25F02AC182F40401300E8227D6
:102C400024EC0EF02BC182F40401300E822724EC18
:102C50000EF02CC182F40401300E822724EC0EF019
:102C60002DC182F40401300E822724EC0EF02EC117
:102C700082F40401300E822724EC0EF02FC182F47E
:102C80000401300E822724EC0EF030C182F40401DE
:102C9000300E822724EC0EF031C182F40401300E94
:102CA000822724EC0EF032C182F40401300E822718
:102CB00024EC0EF033C182F40401300E822724ECA0
:102CC0000EF0C4EF16F00F98D3EC2AF0F8EF1EF0D8
:102CD00004014C0E826F24EC0EF00401350E826F5D
:102CE00024EC0EF004012C0E826F24EC0EF0B9ECF3
:102CF00025F00784B5C500F107945CEC25F031C1DF
:102D000082F40401300E822724EC0EF032C182F4EA
:102D10000401300E822724EC0EF033C182F404014A
:102D2000300E822724EC0EF0C4EF16F096EC2AF059
:102D3000B9EC25F033C500F15CEC25F004014C0E34
:102D4000826F24EC0EF00401360E826F24EC0EF03C
:102D500004012C0E826F24EC0EF031C182F40401C8
:102D6000300E822724EC0EF032C182F40401300EC2
:102D7000822724EC0EF033C182F40401300E822746
:102D800024EC0EF0C4EF16F02EEC0EF0F8EF1EF06F
:102D900004014C0E826F24EC0EF00401500E826F81
:102DA00024EC0EF004012C0E826F24EC0EF085C38F
:102DB0002AF186C32BF187C32CF188C32DF189C377
:102DC0002EF18AC32FF18BC330F18CC331F18DC347
:102DD00032F18EC333F1010107EC26F07EEC25F0D1
:102DE00003018451530A0DE0030184514D0A38E078
:102DF0000401780E826F24EC0EF02EEC0EF0F8EF4A
:102E00001EF00401530E826F24EC0EF0250E0C6EA2
:102E100000C10BF0E9EC0AF0260E0C6E01C10BF0BC
:102E2000E9EC0AF0270E0C6E02C10BF0E9EC0AF097
:102E3000280E0C6E03C10BF0E9EC0AF000C153F54B
:102E400001C154F502C155F503C156F500C157F54E
:102E500001C158F502C159F503C15AF5A5EF17F0A4
:102E600004014D0E826F24EC0EF0290E0C6E00C191
:102E70000BF0E9EC0AF000C15BF500C15CF5A5EFD1
:102E800017F004014C0E826F24EC0EF00401540E76
:102E9000826F24EC0EF004012C0E826F24EC0EF0F5
:102EA00084C32AF185C32BF186C32CF187C32DF18E
:102EB00088C32EF189C32FF18AC330F18BC331F15E
:102EC0008DC332F18EC333F1010107EC26F07EECA5
:102ED00025F00101000E046F000E056F010E066F54
:102EE000000E076FCFEC24F0210E0C6E00C10BF02A
:102EF000E9EC0AF0220E0C6E01C10BF0E9EC0AF0CD
:102F0000230E0C6E02C10BF0E9EC0AF0240E0C6EDD
:102F100003C10BF0E9EC0AF000C15DF501C15EF5FB
:102F200002C15FF503C160F5A5EF17F004014C0E77
:102F3000826F24EC0EF00401490E826F24EC0EF037
:102F400004012C0E826F24EC0EF0250E00EC0BF029
:102F5000E8CF00F1260E00EC0BF0E8CF01F1270ED0
:102F600000EC0BF0E8CF02F1280E00EC0BF0E8CFFC
:102F700003F15CEC25F03FEC23F00401730E826F4B
:102F800024EC0EF004012C0E826F24EC0EF0B9EC50
:102F900025F0290E00EC0BF0E8CF00F15CEC25F0F9
:102FA0003FEC23F00401730E826F24EC0EF0040159
:102FB0002C0E826F24EC0EF057C500F158C501F1BC
:102FC00059C502F15AC503F15CEC25F03FEC23F042
:102FD0000401730E826F24EC0EF004012C0E826F3C
:102FE00024EC0EF0B9EC25F05CC500F15CEC25F0AA
:102FF0003FEC23F004016D0E826F24EC0EF004010F
:103000002C0E826F24EC0EF05DC500F15EC501F15F
:103010005FC502F160C503F113EC1FF004012C0E33
:10302000826F24EC0EF02EEC0EF0F8EF1EF083C34E
:103030002AF184C32BF185C32CF186C32DF187C3FC
:103040002EF188C32FF189C330F18AC331F18BC3CC
:1030500032F18CC333F1010107EC26F07EEC25F050
:10306000160E0C6E00C10BF0E9EC0AF0170E0C6E98
:1030700001C10BF0E9EC0AF0180E0C6E02C10BF066
:10308000E9EC0AF0190E0C6E03C10BF0E9EC0AF042
:1030900000C18AF101C18BF102C18CF103C18DF134
:1030A00000C18EF101C18FF102C190F103C191F114
:1030B000F9EF18F083C32AF184C32BF185C32CF1F7
:1030C00086C32DF187C32EF188C32FF189C330F158
:1030D0008AC331F18BC332F18CC333F1010107ECA8
:1030E00026F07EEC25F000C18AF101C18BF102C10E
:1030F0008CF103C18DF100C18EF101C18FF102C1CC
:1031000090F103C191F1F9EF18F083C32AF184C360
:103110002BF185C32CF186C32DF187C32EF188C313
:103120002FF189C330F18AC331F18CC332F18DC3E1
:1031300033F1010107EC26F07EEC25F00101000ED1
:10314000046F000E056F010E066F000E076FCFECC7
:1031500024F01A0E0C6E00C10BF0E9EC0AF01B0E05
:103160000C6E01C10BF0E9EC0AF01C0E0C6E02C1F2
:103170000BF0E9EC0AF01D0E0C6E03C10BF0E9EC4C
:103180000AF000C192F101C193F102C194F103C1AF
:1031900095F1F9EF18F083C32AF184C32BF185C3AD
:1031A0002CF186C32DF187C32EF188C32FF189C37B
:1031B00030F18AC331F18CC332F18DC333F1010197
:1031C00007EC26F07EEC25F00101000E046F000EE6
:1031D000056F010E066F000E076FCFEC24F000C1E3
:1031E00092F101C193F102C194F103C195F1F9EF9C
:1031F00018F0160E00EC0BF0E8CF00F1170E00EC03
:103200000BF0E8CF01F1180E00EC0BF0E8CF02F163
:10321000190E00EC0BF0E8CF03F15CEC25F03FEC6D
:1032200023F00401730E826F24EC0EF004012C0EC7
:10323000826F24EC0EF08AC100F18BC101F18CC1C8
:1032400002F18DC103F15CEC25F03FEC23F00401A9
:10325000730E826F24EC0EF004012C0E826F24ECAE
:103260000EF01A0E00EC0BF0E8CF00F11B0E00EC94
:103270000BF0E8CF01F11C0E00EC0BF0E8CF02F1EF
:103280001D0E00EC0BF0E8CF03F113EC1FF004016E
:103290002C0E826F24EC0EF092C100F193C101F16B
:1032A00094C102F195C103F113EC1FF02EEC0EF066
:1032B000F8EF1EF00401690E826F24EC0EF0040199
:1032C0002C0E826F24EC0EF00101040E006F000E34
:1032D000016F000E026F000E036F5CEC25F02CC135
:1032E00082F40401300E822724EC0EF02DC182F40A
:1032F0000401300E822724EC0EF02EC182F404016A
:10330000300E822724EC0EF02FC182F40401300E1F
:10331000822724EC0EF030C182F40401300E8227A3
:1033200024EC0EF031C182F40401300E822724EC2B
:103330000EF032C182F40401300E822724EC0EF02C
:1033400033C182F40401300E822724EC0EF0040114
:103350002C0E826F24EC0EF00101060E006F000EA1
:10336000016F000E026F000E036F5CEC25F02CC1A4
:1033700082F40401300E822724EC0EF02DC182F479
:103380000401300E822724EC0EF02EC182F40401D9
:10339000300E822724EC0EF02FC182F40401300E8F
:1033A000822724EC0EF030C182F40401300E822713
:1033B00024EC0EF031C182F40401300E822724EC9B
:1033C0000EF032C182F40401300E822724EC0EF09C
:1033D00033C182F40401300E822724EC0EF0040184
:1033E0002C0E826F24EC0EF00101280E006F000EEF
:1033F000016F000E026F000E036F5CEC25F02CC114
:1034000082F40401300E822724EC0EF02DC182F4E8
:103410000401300E822724EC0EF02EC182F4040148
:10342000300E822724EC0EF02FC182F40401300EFE
:10343000822724EC0EF030C182F40401300E822782
:1034400024EC0EF031C182F40401300E822724EC0A
:103450000EF032C182F40401300E822724EC0EF00B
:1034600033C182F40401300E822724EC0EF00401F3
:103470002C0E826F24EC0EF0200EF86EF76AF66ABE
:1034800004010900F5CF82F424EC0EF00900F5CF19
:1034900082F424EC0EF00900F5CF82F424EC0EF057
:1034A0000900F5CF82F424EC0EF00900F5CF82F488
:1034B00024EC0EF00900F5CF82F424EC0EF00900A4
:1034C000F5CF82F424EC0EF00900F5CF82F424EC61
:1034D0000EF02EEC0EF0F8EF1EF08351630AD8A424
:1034E000F8EF1EF08451610AD8A4F8EF1EF0855160
:1034F0006C0AD8A4F8EF1EF08651410A42E08651CA
:10350000440A1BE08651420AD8B4D4EF1AF086511F
:10351000350AD8B482EF20F08651360AD8B4D7EFF6
:1035200020F08651370AD8B440EF21F08651380A8E
:10353000D8B49EEF21F0F8EF1EF00798079A040127
:103540007A0E826F24EC0EF00401780E826F24EC68
:103550000EF00401640E826F24EC0EF081A8B8EF27
:103560001AF00401550E826F24EC0EF0BDEF1AF034
:1035700004014C0E826F24EC0EF02EEC0EF0F8EFEE
:103580001EF00788079A04017A0E826F24EC0EF071
:103590000401410E826F24EC0EF00401610E826F73
:1035A00024EC0EF0AEEF1AF00798078A04017A0EA9
:1035B000826F24EC0EF00401420E826F24EC0EF0B8
:1035C0000401610E826F24EC0EF0AEEF1AF00101DF
:1035D0006667F2EF1AF06767F2EF1AF06867F2EFCA
:1035E0001AF069670AEF1BF04F67FEEF1AF0506799
:1035F000FEEF1AF05167FEEF1AF052670AEF1BF068
:103600000101000E006F000E016F000E026F000E30
:10361000036F120011B818EF1BF00101620E046F66
:10362000010E056F000E066F000E076F21EF1BF0F5
:103630000101A70E046F020E056F000E066F000E4B
:10364000076F66C100F167C101F168C102F169C18C
:1036500003F1BEEC24F003BF9CEF1BF00101000E50
:10366000046FA80E056F550E066F020E076F66C138
:1036700000F167C101F168C102F169C103F166C1DE
:1036800086F167C187F168C188F169C189F1BEEC33
:1036900024F003BF55EF1BF00101000E866FA80E4A
:1036A000876F550E886F020E896F0E0E00EC0BF0BF
:1036B000E8CF18F10F0E00EC0BF0E8CF19F1100E67
:1036C00000EC0BF0E8CF1AF1110E00EC0BF0E8CF94
:1036D0001BF107EC24F086C104F187C105F188C114
:1036E00006F189C107F1BEEC24F00782CBEC23F090
:1036F00007EC24F00792CBEC23F086C100F187C1E0
:1037000001F188C102F189C103F10792CBEC23F0EA
:10371000CC0E046FE00E056F870E066F050E076F67
:10372000BEEC24F000C118F101C119F102C11AF177
:1037300003C11BF1D4EF1BF00101800E006F1A0EC4
:10374000016F060E026F000E036F4FC104F150C1EE
:1037500005F151C106F152C107F1BEEC24F003AFEF
:10376000B5EF1BF0B9EC25F012000E0E00EC0BF0DB
:10377000E8CF18F10F0E00EC0BF0E8CF19F1100EA6
:1037800000EC0BF0E8CF1AF1110E00EC0BF0E8CFD3
:103790001BF14FC100F150C101F151C102F152C101
:1037A00003F10782CBEC23F018C100F119C101F13C
:1037B0001AC102F11BC103F112000401730E826FE2
:1037C00024EC0EF004012C0E826F24EC0EF0078422
:1037D00062C166F163C167F164C168F165C169F1F5
:1037E0004BC14FF14CC150F14DC151F14EC152F19D
:1037F00057C159F158C15AF1079403EC1CF02EEC53
:103800000EF0F8EF1EF066C100F167C101F168C16A
:1038100002F169C103F101015CEC25F03FEC23F0FA
:103820000401630E826F24EC0EF004012C0E826FF3
:1038300024EC0EF04FC100F150C101F151C102F171
:1038400052C103F101015CEC25F03FEC23F00401CF
:10385000660E826F24EC0EF004012C0E826F24ECB5
:103860000EF0B9EC25F059C100F15AC101F1010186
:103870005CEC25F03FEC23F00401740E826F24EC25
:103880000EF0120010820401530E826F24EC0EF031
:1038900004012C0E826F24EC0EF083C32AF184C342
:1038A0002BF185C32CF186C32DF187C32EF188C37C
:1038B0002FF189C330F18AC331F18BC332F18CC34C
:1038C00033F1010107EC26F07EEC25F000C166F132
:1038D00001C167F102C168F103C169F18EC32AF128
:1038E0008FC32BF190C32CF191C32DF192C32EF114
:1038F00093C32FF194C330F195C331F196C332F1E4
:1039000097C333F1010107EC26F07EEC25F000C1EE
:103910004FF101C150F102C151F103C152F1FAEC72
:1039200025F099C32FF19AC330F19BC331F19CC3A9
:1039300032F19DC333F1010107EC26F07EEC25F056
:1039400000C159F101C15AF103EC1CF004012C0E25
:10395000826F24EC0EF0B4EF1CF08251520A03E1A6
:103960000F82B4EF1CF00F928251750A03E11084AC
:10397000BBEF1CF0109411A0C2EF1CF011A4C2EF19
:103980001CF010848251550A03E11086C9EF1CF027
:103990001096078410B226EF1DF010A412EF1DF050
:1039A000B6C166F1B7C167F1B8C168F1B9C169F1D3
:1039B000BAC16AF1BBC16BF1BCC16CF1BDC16DF1A3
:1039C000BEC16EF1BFC16FF1C0C170F1C1C171F173
:1039D000C2C172F1C3C173F1C4C174F1C5C175F143
:1039E000C6C176F1C7C177F1C8C178F1C9C179F113
:1039F000CAC17AF1CBC17BF1CCC17CF1CDC17DF1E3
:103A0000CEC17EF1CFC17FF1D0C180F1D1C181F1B2
:103A1000D2C182F1D3C183F1D4C184F1D5C185F182
:103A20001AEF1DF062C166F163C167F164C168F10C
:103A300065C169F14BC14FF14CC150F14DC151F11C
:103A40004EC152F157C159F158C15AF107940FA014
:103A500048EF1DF00101926735EF1DF0936735EFD8
:103A60001DF0946735EF1DF0956739EF1DF048EFB5
:103A70001DF0E7EC1AF092C104F193C105F194C175
:103A800006F195C107F1BEEC24F003BFBEEF1EF0B6
:103A9000E7EC1AF00101000E046F000E056F010E35
:103AA000066F000E076FEFEC24F011A087EF1DF0FA
:103AB00011A287EF1DF05CEC25F0296762EF1DF085
:103AC00069EF1DF004012D0E826F24EC0EF0BCEFA7
:103AD0001EF030C182F40401300E822724EC0EF077
:103AE00031C182F40401300E822724EC0EF032C181
:103AF00082F40401300E822724EC0EF033C182F4EC
:103B00000401300E822724EC0EF0BCEF1EF010A44E
:103B100091EF1DF00401750E826F24EC0EF096EF0C
:103B20001DF00401720E826F24EC0EF004012C0EC5
:103B3000826F24EC0EF05CEC25F02967A5EF1DF0F8
:103B40000401200E826FA8EF1DF004012D0E826F7C
:103B500024EC0EF030C182F40401300E822724ECF4
:103B60000EF031C182F40401300E822724EC0EF0F5
:103B700004012E0E826F24EC0EF032C182F4040197
:103B8000300E822724EC0EF033C182F40401300E93
:103B9000822724EC0EF004016D0E826F24EC0EF0EF
:103BA00004012C0E826F24EC0EF04FC100F150C1C5
:103BB00001F151C102F152C103F101015CEC25F0A8
:103BC0003FEC23F00401480E826F24EC0EF0040158
:103BD0007A0E826F24EC0EF004012C0E826F24EC1E
:103BE0000EF066C100F167C101F168C102F169C15F
:103BF00003F101015CEC25F03FEC23F00401630EBE
:103C0000826F24EC0EF004012C0E826F24EC0EF077
:103C100066C100F167C101F168C102F169C103F138
:103C200001010A0E046F000E056F000E066F000EF4
:103C3000076FCFEC24F0000E046F120E056F000E1C
:103C4000066F000E076FEFEC24F05CEC25F02AC144
:103C500082F40401300E822724EC0EF02BC182F492
:103C60000401300E822724EC0EF02CC182F40401F2
:103C7000300E822724EC0EF02DC182F40401300EA8
:103C8000822724EC0EF02EC182F40401300E82272C
:103C900024EC0EF02FC182F40401300E822724ECB4
:103CA0000EF030C182F40401300E822724EC0EF0B5
:103CB00004012E0E826F24EC0EF031C182F4040157
:103CC000300E822724EC0EF032C182F40401300E53
:103CD000822724EC0EF033C182F40401300E8227D7
:103CE00024EC0EF00401730E826F24EC0EF004013C
:103CF0002C0E826F24EC0EF0B9EC25F059C100F1C6
:103D00005AC101F122EC20F00FB28AEF1EF00FA091
:103D1000BCEF1EF004012C0E826F24EC0EF0200E7E
:103D2000F86EF76AF66A04010900F5CF82F424EC14
:103D30000EF00900F5CF82F424EC0EF00900F5CF67
:103D400082F424EC0EF00900F5CF82F424EC0EF09E
:103D50000900F5CF82F424EC0EF00900F5CF82F4CF
:103D600024EC0EF00900F5CF82F424EC0EF00900EB
:103D7000F5CF82F424EC0EF02EEC0EF00F90F8EF5D
:103D80001EF00401630E826F24EC0EF004012C0E71
:103D9000826F24EC0EF0FEEC1EF004012C0E826FFC
:103DA00024EC0EF071EC1FF004012C0E826F24EC59
:103DB0000EF0EDEC1FF004012C0E826F24EC0EF0DF
:103DC0000101F80E006FCD0E016F660E026F030E3B
:103DD000036F13EC1FF004012C0E826F24EC0EF025
:103DE00003EC20F02EEC0EF0F8EF1EF02EEC0EF0AF
:103DF0000301C26B0790109207EF22F0D8900E0ECD
:103E000000EC0BF0E8CF00F10F0E00EC0BF0E8CF68
:103E100001F1100E00EC0BF0E8CF02F1110E00ECF6
:103E20000BF0E8CF03F10101000E046F000E056FE7
:103E3000010E066F000E076FEFEC24F05CEC25F02E
:103E40002AC182F40401300E822724EC0EF02BC12B
:103E500082F40401300E822724EC0EF02CC182F48F
:103E60000401300E822724EC0EF02DC182F40401EF
:103E7000300E822724EC0EF02EC182F40401300EA5
:103E8000822724EC0EF02FC182F40401300E822729
:103E900024EC0EF030C182F40401300E822724ECB1
:103EA0000EF031C182F40401300E822724EC0EF0B2
:103EB00004012E0E826F24EC0EF032C182F4040154
:103EC000300E822724EC0EF033C182F40401300E50
:103ED000822724EC0EF004016D0E826F24EC0EF0AC
:103EE0001200120E00EC0BF0E8CF00F1130E00EC04
:103EF0000BF0E8CF01F1140E00EC0BF0E8CF02F16B
:103F0000150E00EC0BF0E8CF03F101010A0E046F6F
:103F1000000E056F000E066F000E076FCFEC24F049
:103F2000000E046F120E056F000E066F000E076F75
:103F3000EFEC24F05CEC25F02AC182F40401300E91
:103F4000822724EC0EF02BC182F40401300E82276C
:103F500024EC0EF02CC182F40401300E822724ECF4
:103F60000EF02DC182F40401300E822724EC0EF0F5
:103F70002EC182F40401300E822724EC0EF02FC1F2
:103F800082F40401300E822724EC0EF030C182F45A
:103F90000401300E822724EC0EF004012E0E826FF5
:103FA00024EC0EF031C182F40401300E822724EC9F
:103FB0000EF032C182F40401300E822724EC0EF0A0
:103FC00033C182F40401300E822724EC0EF0040188
:103FD000730E826F24EC0EF012000A0E00EC0BF050
:103FE000E8CF00F10B0E00EC0BF0E8CF01F10C0E66
:103FF00000EC0BF0E8CF02F10D0E00EC0BF0E8CF77
:1040000003F122EF20F0060E00EC0BF0E8CF00F1F8
:10401000070E00EC0BF0E8CF01F1080E00EC0BF0FE
:10402000E8CF02F1090E00EC0BF0E8CF03F122EF2C
:1040300020F00101B9EC25F0078457C100F158C107
:1040400001F107940101E80E046F800E056F000E68
:10405000066F000E076FCFEC24F0000E046F040E05
:10406000056F000E066F000E076FEFEC24F0880E50
:10407000046F130E056F000E066F000E076FBEEC87
:1040800024F00A0E046F000E056F000E066F000E7E
:10409000076FEFEC24F05CEC25F00101296756EF87
:1040A00020F00401200E826F59EF20F004012D0E44
:1040B000826F24EC0EF030C182F40401300E8227AE
:1040C00024EC0EF031C182F40401300E822724EC7E
:1040D0000EF032C182F40401300E822724EC0EF07F
:1040E00004012E0E826F24EC0EF033C182F4040121
:1040F000300E822724EC0EF00401430E826F24EC74
:104100000EF0120087C32AF188C32BF189C32CF16A
:104110008AC32DF18BC32EF18CC32FF18DC330F1E7
:104120008EC331F190C332F191C333F10101296B98
:1041300007EC26F07EEC25F00101000E046F000E66
:10414000056F010E066F000E076FCFEC24F00E0E08
:104150000C6E00C10BF0E9EC0AF00F0E0C6E01C101
:104160000BF0E9EC0AF0100E0C6E02C10BF0E9EC5A
:104170000AF0110E0C6E03C10BF0E9EC0AF0040119
:104180007A0E826F24EC0EF004012C0E826F24EC68
:104190000EF00401350E826F24EC0EF004012C0E9B
:1041A000826F24EC0EF0FEEC1EF0BDEF1AF087C318
:1041B0002AF188C32BF189C32CF18AC32DF18BC35B
:1041C0002EF18CC32FF18DC330F18EC331F190C32A
:1041D00032F191C333F10101296B07EC26F07EEC3B
:1041E00025F0880E046F130E056F000E066F000E8B
:1041F000076FC3EC24F0000E046F040E056F000E71
:10420000066F000E076FCFEC24F00101E80E046F7B
:10421000800E056F000E066F000E076FEFEC24F0A6
:104220000A0E0C6E00C10BF0E9EC0AF00B0E0C6EDE
:1042300001C10BF0E9EC0AF00C0E0C6E02C10BF0A0
:10424000E9EC0AF00D0E0C6E03C10BF0E9EC0AF07C
:1042500004017A0E826F24EC0EF004012C0E826FA2
:1042600024EC0EF00401360E826F24EC0EF00401F3
:104270002C0E826F24EC0EF0EDEC1FF0BDEF1AF067
:1042800087C32AF188C32BF189C32CF18AC32DF18E
:104290008BC32EF18CC32FF18DC330F18FC331F15D
:1042A00090C332F191C333F1010107EC26F07EECAB
:1042B00025F0000E046F120E056F000E066F000E43
:1042C000076FCFEC24F001010A0E046F000E056F9A
:1042D000000E066F000E076FEFEC24F0120E0C6E4E
:1042E00000C10BF0E9EC0AF0130E0C6E01C10BF0EB
:1042F000E9EC0AF0140E0C6E02C10BF0E9EC0AF0C6
:10430000150E0C6E03C10BF0E9EC0AF004017A0EF5
:10431000826F24EC0EF004012C0E826F24EC0EF060
:104320000401370E826F24EC0EF004012C0E826F14
:1043300024EC0EF071EC1FF0BDEF1AF087C32AF1E8
:1043400088C32BF189C32CF18AC32DF18BC32EF1C5
:104350008CC32FF18DC330F18EC331F190C332F194
:1043600091C333F10101296B07EC26F07EEC25F0B7
:10437000880E046F130E056F000E066F000E076F98
:10438000C3EC24F0000E046F040E056F000E066FE0
:10439000000E076FCFEC24F00101E80E046F800ED1
:1043A000056F000E066F000E076FEFEC24F0060E8F
:1043B0000C6E00C10BF0E9EC0AF0070E0C6E01C1A7
:1043C0000BF0E9EC0AF0080E0C6E02C10BF0E9EC00
:1043D0000AF0090E0C6E03C10BF0E9EC0AF00401BF
:1043E0007A0E826F24EC0EF004012C0E826F24EC06
:1043F0000EF00401380E826F24EC0EF004012C0E36
:10440000826F24EC0EF003EC20F0BDEF1AF081A8CF
:10441000C5EF22F007A87EEF22F00101800E006FA9
:104420001A0E016F060E026F000E036F4BC104F1EE
:104430004CC105F14DC106F14EC107F1BEEC24F0AF
:1044400003BFC5EF22F039EC23F04BC100F14CC1A2
:1044500001F14DC102F14EC103F10782CBEC23F013
:1044600018C104F119C105F11AC106F11BC107F108
:10447000F80E006FCD0E016F660E026F030E036F14
:10448000BEEC24F00E0E0C6E00C10BF0E9EC0AF04D
:104490000F0E0C6E01C10BF0E9EC0AF0100E0C6E61
:1044A00002C10BF0E9EC0AF0110E0C6E03C10BF027
:1044B000E9EC0AF007840101B9EC25F057C100F1DD
:1044C00058C101F107940A0E0C6E00C10BF0E9EC23
:1044D0000AF00B0E0C6E01C10BF0E9EC0AF00C0EA9
:1044E0000C6E02C10BF0E9EC0AF00D0E0C6E03C16C
:1044F0000BF0E9EC0AF00798C5EF22F007AAC5EF28
:1045000022F007840101B9EC25F057C100F158C130
:1045100001F10794060E0C6E00C10BF0E9EC0AF0F5
:10452000070E0C6E01C10BF0E9EC0AF0080E0C6EE0
:1045300002C10BF0E9EC0AF0090E0C6E03C10BF09E
:10454000E9EC0AF0078462C100F163C101F164C1C2
:1045500002F165C103F10794120E0C6E00C10BF05D
:10456000E9EC0AF0130E0C6E01C10BF0E9EC0AF055
:10457000140E0C6E02C10BF0E9EC0AF0150E0C6E75
:1045800003C10BF0E9EC0AF0079A0401805181198C
:104590007F0B0BE09EA809D014EE00F081517F0B39
:1045A000E126E750812B0F01AD6E05012F51010A65
:1045B00013E081AAECEF22F005012F51000A0AE076
:1045C0000FB8ECEF22F005013067ECEF22F00FB8E6
:1045D000ECEF22F05BEF2CF081B801EF23F0E9EC77
:1045E00026F005012F51020A02E001EF23F05C2FB3
:1045F00001EF23F05BC55CF50501010E306F3C0E49
:10460000316F83EF0DF018C100F119C101F11AC12A
:1046100002F11BC103F1000E046F000E056F010EC5
:10462000066F000E076FEFEC24F029A12EEF23F0A8
:104630002051D8B42EEF23F018C100F119C101F1B7
:104640001AC102F11BC103F1000E046F000E056FC9
:104650000A0E066F000E076FEFEC24F01200010146
:10466000045100130551011306510213075103139E
:1046700012000101186B196B1A6B1B6B12002AC117
:1046800082F40401300E822724EC0EF02BC182F458
:104690000401300E822724EC0EF02CC182F40401B8
:1046A000300E822724EC0EF02DC182F40401300E6E
:1046B000822724EC0EF02EC182F40401300E8227F2
:1046C00024EC0EF02FC182F40401300E822724EC7A
:1046D0000EF030C182F40401300E822724EC0EF07B
:1046E00031C182F40401300E822724EC0EF032C175
:1046F00082F40401300E822724EC0EF033C182F4E0
:104700000401300E822724EC0EF012002FC182F437
:104710000401300E822724EC0EF030C182F4040133
:10472000300E822724EC0EF031C182F40401300EE9
:10473000822724EC0EF032C182F40401300E82276D
:1047400024EC0EF033C182F40401300E822724ECF5
:104750000EF01200060E126E060E136E060E146E8A
:10476000122EB0EF23F0132EB0EF23F0142EB0EF83
:1047700023F08B84020E126E020E136E020E146E64
:10478000122EC0EF23F0132EC0EF23F0142EC0EF33
:1047900023F08B9412000101005305E1015303E162
:1047A000025301E1002B8EEC24F0B9EC25F03951D5
:1047B000006F3A51016F420E046F4B0E056F000EF1
:1047C000066F000E076FCFEC24F000C104F101C1A9
:1047D00005F102C106F103C107F118C100F119C1C9
:1047E00001F11AC102F11BC103F107B2FCEF23F082
:1047F000C3EC24F0FEEF23F0BEEC24F000C118F16E
:1048000001C119F102C11AF103C11BF11200B9EC87
:1048100025F059C100F15AC101F1060E00EC0BF070
:10482000E8CF04F1070E00EC0BF0E8CF05F1080E1D
:1048300000EC0BF0E8CF06F1090E00EC0BF0E8CF2E
:1048400007F1BEEC24F000C124F101C125F102C141
:1048500026F103C127F1290E046F000E056F000E2B
:10486000066F000E076FCFEC24F0EE0E046F430EC0
:10487000056F000E066F000E076FC3EC24F024C115
:1048800004F125C105F126C106F127C107F1CFECDE
:1048900024F000C11CF101C11DF102C11EF103C1D0
:1048A0001FF1120E00EC0BF0E8CF04F1130E00EC38
:1048B0000BF0E8CF05F1140E00EC0BF0E8CF06F199
:1048C000150E00EC0BF0E8CF07F10D0E006F000E97
:1048D000016F000E026F000E036FCFEC24F0180E74
:1048E000046F000E056F000E066F000E076FEFECF1
:1048F00024F01CC104F11DC105F11EC106F11FC148
:1049000007F1C3EC24F06A0E046F2A0E056F000E47
:10491000066F000E076FBEEC24F01200BF0EFA6E99
:10492000200E3A6F396BD8900037013702370337C2
:10493000D8B09FEF24F03A2F94EF24F039073A07CC
:104940000353D8B412000331070B80093F6F0339BA
:104950000F0B010F396F80EC5FF0406F390580EC71
:104960005FF0405D405F396B3F33D8B03927393352
:104970003FA9B4EF24F04051392712000101DEECC9
:1049800025F0D8B01200010103510719346FA1ECD2
:1049900025F0D8900751031934AF800F12000101A0
:1049A000346BC5EC25F0D8A0DBEC25F0D8B01200B4
:1049B000B0EC25F0B9EC25F01F0E366FF1EC25F0C8
:1049C0000B35D8B0A1EC25F0D8A00335D8B0120033
:1049D000362FDEEF24F034B1C8EC25F012000101CF
:1049E000346B04510511061107110008D8A0C5EC5D
:1049F00025F0D8A0DBEC25F0D8B01200086B096BCD
:104A00000A6B0B6BF1EC25F01F0E366FF1EC25F005
:104A100007510B5DD8A419EF25F006510A5DD8A403
:104A200019EF25F00551095DD8A419EF25F00451BF
:104A3000085DD8A02CEF25F00451085F0551D8A0DF
:104A4000053D095F0651D8A0063D0A5F0751D8A071
:104A5000073D0B5FD8900081362F06EF25F034B16B
:104A6000C8EC25F0346BC5EC25F0D890F5EC25F0BA
:104A700007510B5DD8A449EF25F006510A5DD8A473
:104A800049EF25F00551095DD8A449EF25F00451FF
:104A9000085DD8A058EF25F0003F58EF25F0013F02
:104AA00058EF25F0023F58EF25F0032BD8B4120041
:104AB00034B1C8EC25F012000101346BC5EC25F0CF
:104AC000D8B01200FAEC25F0200E366F003701370F
:104AD0000237033711EE33F00A0E376FE7360A0E4E
:104AE000E75CD8B0E76EE552372F6EEF25F0362F32
:104AF00066EF25F034B12981D890120001010A0E29
:104B0000346F200E366F11EE29F03451376F0A0ED4
:104B1000D890E652D8B0E726E732372F89EF25F054
:104B20000333023301330033362F83EF25F0E75090
:104B3000FF0FD8A00335D8B0120029B1C8EC25F07A
:104B40001200045100270551D8B0053D0127065138
:104B5000D8B0063D02270751D8B0073D0327120001
:104B60000051086F0151096F02510A6F03510B6F19
:104B700012000101006B016B026B036B120001015B
:104B8000046B056B066B076B12000335D8A012008F
:104B90000351800B001F011F021F031F003FD8EFAE
:104BA00025F0013FD8EF25F0023FD8EF25F0032B89
:104BB000342B032512000735D8A012000751800BB3
:104BC000041F051F061F071F043FEEEF25F0053FDA
:104BD000EEEF25F0063FEEEF25F0072B342B0725EF
:104BE00012000037013702370337083709370A3711
:104BF0000B3712000101296B2A6B2B6B2C6B2D6B71
:104C00002E6B2F6B306B316B326B336B12000101EB
:104C10002A510F0B2A6F2B510F0B2B6F2C510F0B9F
:104C20002C6F2D510F0B2D6F2E510F0B2E6F2F51FF
:104C30000F0B2F6F30510F0B306F31510F0B316F46
:104C400032510F0B326F33510F0B336F120010A81C
:104C500006D08994000EC76E220EC66E05D08984D8
:104C6000000EC76E220EC66E050EE82EFED712008D
:104C700010A802D0898401D08994050EE82EFED7B1
:104C8000120027EC26F09E96C69E000EC96EFF0EFF
:104C90009EB602D0E82EFCD79E96C69E000EC96E28
:104CA000FF0E9EB602D0E82EFCD7C9CFABF59E967C
:104CB000C69E000EC96EFF0E9EB602D0E82EFCD72F
:104CC000C9CFACF59E96C69E000EC96EFF0E9EB66D
:104CD00002D0E82EFCD7C9CFADF59E96C69E000E39
:104CE000C96EFF0E9EB602D0E82EFCD7C9CFAEF536
:104CF0009E96C69E000EC96EFF0E9EB602D0E82E8E
:104D0000FCD7C9CFAFF59E96C69E000EC96EFF0EAA
:104D10009EB602D0E82EFCD7C9CFB0F59E96C69EAF
:104D2000000EC96EFF0E9EB602D0E82EFCD7C9CF8A
:104D3000B1F538EC26F0120027EC26F09E96C69EC0
:104D4000800EC96EFF0E9EB602D0E82EFCD79E964E
:104D5000C69EABC5C9FFFF0E9EB602D0E82EFCD79B
:104D60009E96C69EACC5C9FFFF0E9EB602D0E82E29
:104D7000FCD79E96C69EADC5C9FFFF0E9EB602D05B
:104D8000E82EFCD79E96C69EAEC5C9FFFF0E9EB606
:104D900002D0E82EFCD79E96C69EAFC5C9FFFF0E77
:104DA0009EB602D0E82EFCD79E96C69EB0C5C9FF1F
:104DB000FF0E9EB602D0E82EFCD79E96C69EB1C5C9
:104DC000C9FFFF0E9EB602D0E82EFCD738EC26F0C5
:104DD000120027EC26F09E96C69E070EC96EFF0EA7
:104DE0009EB602D0E82EFCD79E96C69E000EC96ED7
:104DF000FF0E9EB602D0E82EFCD7C9CFABF59E962B
:104E0000C69E000EC96EFF0E9EB602D0E82EFCD7DD
:104E1000C9CFACF59E96C69E000EC96EFF0E9EB61B
:104E200002D0E82EFCD7C9CFADF59E96C69E000EE7
:104E3000C96EFF0E9EB602D0E82EFCD7C9CFAEF5E4
:104E400038EC26F027EC26F09E96C69E16C0C9FFC9
:104E5000FF0E9EB602D0E82EFCD79E96C69E000E90
:104E6000C96EFF0E9EB602D0E82EFCD7C9CFB2F5B0
:104E700038EC26F0120027EC26F09E96C69E870E90
:104E8000C96EFF0E9EB602D0E82EFCD79E96C69E37
:104E9000ABC5C9FFFF0E9EB602D0E82EFCD79E968A
:104EA000C69EACC5C9FFFF0E9EB602D0E82EFCD749
:104EB0009E96C69EADC5C9FFFF0E9EB602D0E82ED7
:104EC000FCD79E96C69EAEC5C9FFFF0E9EB602D009
:104ED000E82EFCD738EC26F027EC26F09E96C69EEE
:104EE00017C0C9FFFF0E9EB602D0E82EFCD79E96D3
:104EF000C69EB2C5C9FFFF0E9EB602D0E82EFCD7F3
:104F000038EC26F0120027EC26F09E96C69E870EFF
:104F1000C96EFF0E9EB602D0E82EFCD79E96C69EA6
:104F2000000EC96EFF0E9EB602D0E82EFCD79E96EC
:104F3000C69E800EC96EFF0E9EB602D0E82EFCD72C
:104F40009E96C69E800EC96EFF0E9EB602D0E82EBB
:104F5000FCD79E96C69E800EC96EFF0E9EB602D0EE
:104F6000E82EFCD738EC26F0120027EC26F09E96AF
:104F7000C69E870EC96EFF0E9EB602D0E82EFCD7E5
:104F80009E96C69E000EC96EFF0E9EB602D0E82EFB
:104F9000FCD79E96C69E000EC96EFF0E9EB602D02E
:104FA000E82EFCD79E96C69E800EC96EFF0E9EB65A
:104FB00002D0E82EFCD79E96C69E800EC96EFF0ECC
:104FC0009EB602D0E82EFCD738EC26F0120010A8CE
:104FD0002DD027EC26F09E96C69E17C0C9FFFF0E67
:104FE0009EB602D0E82EFCD79E96C69E450EC96E90
:104FF000FF0E9EB602D0E82EFCD738EC26F027EC48
:1050000026F09E96C69E8F0EC96EFF0E9EB602D0EB
:10501000E82EFCD79E96C69E000EC96EFF0E9EB669
:1050200002D0E82EFCD738EC26F0120027EC26F050
:105030009E96C69E17C0C9FFFF0E9EB602D0E82EF0
:10504000FCD79E96C69E010EC96EFF0E9EB602D07C
:10505000E82EFCD738EC26F027EC26F09E96C69E6C
:10506000910EC96EFF0E9EB602D0E82EFCD79E961A
:10507000C69EA50EC96EFF0E9EB602D0E82EFCD7C6
:1050800038EC26F0120027EC26F09E96C69E17C03C
:10509000C9FFFF0E9EB602D0E82EFCD79E96C69E94
:1050A000810EC96EFF0E9EB602D0E82EFCD738ECFA
:1050B00026F0120027EC26F09E96C69E17C0C9FF68
:1050C000FF0E9EB602D0E82EFCD79E96C69E010E1D
:1050D000C96EFF0E9EB602D0E82EFCD738EC26F043
:1050E000120027EC26F09E96C69E910EC96EFF0E0A
:1050F0009EB602D0E82EFCD79E96C69EA50EC96E1F
:10510000FF0E9EB602D0E82EFCD738EC26F0120037
:1051100027EC26F09E96C69E910EC96EFF0E9EB697
:1051200002D0E82EFCD79E96C69E000EC96EFF0EDA
:105130009EB602D0E82EFCD738EC26F0120005010E
:10514000256B266B276B286B899A400EC76E200E45
:10515000C66E9E96C69E030EC96EFF0E9EB602D008
:10516000E82EFCD79E96C69E27C5C9FFFF0E9EB6A9
:1051700002D0E82EFCD79E96C69E26C5C9FFFF0E1C
:105180009EB602D0E82EFCD79E96C69E25C5C9FFC6
:10519000FF0E9EB602D0E82EFCD79E96C69EC95240
:1051A000FF0E9EB602D0E82EFCD7898A0F01C950A7
:1051B000FF0A01E1120005012E51130A05E0050165
:1051C0002E51170A0CE012000501F00E256FFF0E9C
:1051D000266F0F0E276F000E286FF8EF28F00501DD
:1051E000F00E256FFF0E266FFF0E276F000E286F43
:1051F000899A400EC76E200EC66E9E96C69E030EFE
:10520000C96EFF0E9EB602D0E82EFCD79E96C69EB3
:1052100027C5C9FFFF0E9EB602D0E82EFCD79E968A
:10522000C69E26C5C9FFFF0E9EB602D0E82EFCD74B
:105230009E96C69E25C5C9FFFF0E9EB602D0E82EDB
:10524000FCD79E96C69EC952FF0E9EB602D0E82E8F
:10525000FCD7898A0F01C950FF0A1DE005012E51B4
:10526000130A05E005012E51170A0BE01200050193
:10527000000E256F000E266F100E276F000E286F90
:1052800012000501000E256F000E266F000E276F1D
:10529000010E286F12000501256B266B276B286B0A
:1052A00005012E51130A05E005012E51170A0CE0E5
:1052B00012000501000E216F000E226F080E236FF1
:1052C000000E246F6DEF29F00501000E216F000E16
:1052D000226F800E236F000E246F21C500F122C5BE
:1052E00001F123C502F124C503F125C504F126C54A
:1052F00005F127C506F128C507F12FEC23F000C101
:1053000025F501C126F502C127F503C128F5899AC3
:10531000400EC76E200EC66E9E96C69E030EC96EC8
:10532000FF0E9EB602D0E82EFCD79E96C69E27C5DD
:10533000C9FFFF0E9EB602D0E82EFCD79E96C69EF1
:1053400026C5C9FFFF0E9EB602D0E82EFCD79E965A
:10535000C69E25C5C9FFFF0E9EB602D0E82EFCD71B
:105360009E96C69EC952FF0E9EB602D0E82EFCD76E
:10537000898AC950FF0A08E104C125F505C126F54F
:1053800006C127F507C128F5D8900501243323333A
:10539000223321332151F00B216F2167D7EF29F000
:1053A0002267D7EF29F02367D7EF29F024676DEF45
:1053B00029F00501100E2527E86A2623E86A27232D
:1053C000E86A28231200E86A05012E51130A06E054
:1053D00005012E51170A0BE0020E1200050128519B
:1053E000000A03E12751F00B07E0010E120005014E
:1053F0002851000A01E0010E120029C500F12AC55A
:1054000001F12BC502F12CC503F125C504F126C518
:1054100005F127C506F128C507F1BEEC24F003BF4E
:105420001200E3EC29F0D8A475EF2AF0899A400E17
:10543000C76E200EC66E9E96C69E060EC96EFF0EE5
:105440009EB602D0E82EFCD7898A899A9E96C69E7F
:10545000020EC96EFF0E9EB602D0E82EFCD79E96B5
:10546000C69E27C5C9FFFF0E9EB602D0E82EFCD708
:105470009E96C69E26C5C9FFFF0E9EB602D0E82E98
:10548000FCD79E96C69E25C5C9FFFF0E9EB602D0CC
:10549000E82EFCD79E96C69E000EC96EFF0E9EB6E5
:1054A00002D0E82EFCD7898A899A9E96C69E050E60
:1054B000C96EFF0E9EB602D0E82EFCD79E96C69E01
:1054C000C952FF0E9EB602D0E82EFCD7C9B05EEFDF
:1054D0002AF0898A0501100E2527E86A2623E86A42
:1054E0002723E86A2823FDEF29F01200899A400E4D
:1054F000C76E200EC66E9E96C69E060EC96EFF0E25
:105500009EB602D0E82EFCD7898A899A9E96C69EBE
:10551000C70EC96EFF0E9EB602D0E82EFCD7898A50
:105520000501256B266B276B286B1200899A400EAC
:10553000C76E200EC66E9E96C69E050EC96EFF0EE5
:105540009EB602D0E82EFCD79E96C69EC952FF0E8C
:105550009EB602D0E82EFCD7C9CF33F5898A120057
:10556000899A400EC76E200EC66E9E96C69EB90ED4
:10557000C96EFF0E9EB602D0E82EFCD7898A1200B3
:10558000899A400EC76E200EC66E9E96C69EAB0EC2
:10559000C96EFF0E9EB602D0E82EFCD7898AFF0E98
:1055A000E82EFED71200E3EC29F0D8A41200899A65
:1055B000400EC76E200EC66E9E96C69E030EC96E26
:1055C000FF0E9EB602D0E82EFCD79E96C69E27C53B
:1055D000C9FFFF0E9EB602D0E82EFCD79E96C69E4F
:1055E00026C5C9FFFF0E9EB602D0E82EFCD79E96B8
:1055F000C69E25C5C9FFFF0E9EB602D0E82EFCD779
:105600009E96C69EC952FF0E9EB602D0E82EFCD7CB
:10561000898A0F01C950FF0AD8A4CEEF2BF00501EB
:10562000FE0E336F41EC26F0ABC534F5ACC535F555
:10563000ADC536F5AEC537F5AFC538F5B0C539F5EA
:10564000B1C53AF50784B6C166F1B7C167F1B8C113
:1056500068F1B9C169F14BC14FF14CC150F14DC175
:1056600051F14EC152F157C159F158C15AF1E7EC0D
:105670001AF000C13BF501C13CF502C13DF503C183
:105680003EF505015D674CEF2BF05E674CEF2BF0AC
:105690005F674CEF2BF0606750EF2BF05DEF2BF066
:1056A0005DC504F15EC505F15FC506F160C507F192
:1056B000BEEC24F003BFCEEF2BF059C13FF55AC129
:1056C00040F5B5C541F5B6C542F507940501110E83
:1056D000326F899A400EC76E200EC66E9E96C69E89
:1056E000060EC96EFF0E9EB602D0E82EFCD7898A40
:1056F000899A9E96C69E020EC96EFF0E9EB602D075
:10570000E82EFCD79E96C69E27C5C9FFFF0E9EB603
:1057100002D0E82EFCD79E96C69E26C5C9FFFF0E76
:105720009EB602D0E82EFCD79E96C69E25C5C9FF20
:10573000FF0E9EB602D0E82EFCD725EE33F0322FB6
:1057400002D0AEEF2BF09E96C69EDECFC9FFFF0EB5
:105750009EB602D0E82EFCD79FEF2BF0898A899A5B
:105760009E96C69E050EC96EFF0E9EB602D0E82E0E
:10577000FCD79E96C69EC952FF0E9EB602D0E82E5A
:10578000FCD7C9B0B9EF2BF0898A0501100E252787
:10579000E86A2623E86A2723E86A2823120021C53D
:1057A00000F122C501F123C502F124C503F1899A54
:1057B000400EC76E200EC66E9E96C69E0B0EC96E1C
:1057C000FF0E9EB602D0E82EFCD79E96C69E02C162
:1057D000C9FFFF0E9EB602D0E82EFCD79E96C69E4D
:1057E00001C1C9FFFF0E9EB602D0E82EFCD79E96DF
:1057F000C69E00C1C9FFFF0E9EB602D0E82EFCD7A0
:105800009E96C69EC952FF0E9EB602D0E82EFCD7C9
:1058100025EE33F00501100E326F9E96C69EC952DA
:10582000FF0E9EB602D0E82EFCD7C9CFDEFF322F86
:105830000DEF2CF0898A1200899A400EC76E200E57
:10584000C66E9E96C69E900EC96EFF0E9EB602D084
:10585000E82EFCD79E96C69E000EC96EFF0E9EB621
:1058600002D0E82EFCD79E96C69E000EC96EFF0E93
:105870009EB602D0E82EFCD79E96C69E000EC96E3C
:10588000FF0E9EB602D0E82EFCD79E96C69EC95249
:10589000FF0E9EB602D0E82EFCD7C9CF2DF59E96FE
:1058A000C69EC952FF0E9EB602D0E82EFCD7C9CFC5
:1058B0002EF5898A1200AAEC23F0B5C5E8FFD708B7
:1058C00002E3AAEC23F0B5C5E8FFC80802E3AAEC9E
:1058D00023F0B5C5E8FFB90802E3AAEC23F0B5C58B
:1058E000E8FFAA0802E3AAEC23F0B5C5E8FF9B088D
:1058F00002E3AAEC23F0E9EC26F0B0EC2AF0F29CEB
:10590000F29E8B94C69AC2909482948C720ED36E3F
:10591000D3A4FED789968A909390FF0EE8CF00F02B
:10592000E82EFED7002EFCD78150F294F29A9E907A
:105930009D909E929D92F298F292F290F286F28E53
:045940000300FF0061
:10BF0000E844F926000C160C2B0C3F0C520C640C68
:10BF1000760C860C960CA50CB30CC10CCF0CDC0C6B
:06BF2000E80CF40C000C1B
:00000001FF
